:1000000030C04AC049C048C047C046C045C044C0CF
:1000100043C0E7C041C0A3C13FC03EC03DC03CC0DB
:100020003BC0FFC011C125C137C146C15AC173C110
:100030007AC1FEFEFEFEFEFEFEAABA57BE75FE5750
:10004000AADDAA55AA55AF57BE5F01000100010104
:100050000000010100080101000100000000820011
:10006000F00011241FBECFE5D2E0DEBFCDBF10E00F
:10007000A0E6B0E0E4EFF7E002C005900D92A636EE
:10008000B107D9F710E0A6E6B0E001C01D92A93A89
:10009000B107E1F702D0ACC3B3CFF8948FEF8ABBBE
:1000A0001BBA8F9A309A14BA85BBD4D210927000C2
:1000B00078948091700080FF0CC0809170008E7FDA
:1000C00080937000809168008F3710F0979801C07E
:1000D000979A84D1EECF9C01E199FECF3FBB2EBB16
:1000E000E09A8DB308959C01E199FECF3FBB2EBBF2
:1000F0006DBB0FB6F894E29AE19A0FBE0895809115
:1001000074008F3F09F441C0929AE1E7F0E0A0E665
:10011000B0E0818583838D918187319680E0A6361A
:10012000B807B9F78CEC8093710081E0809372007E
:1001300090918800985E9093730010928200809155
:1001400085008F5F8093850040E050E020E030E044
:1001500008C0F901EF58FF4F8081480F511D2F5FF4
:100160003F4F2917B0F3E92FF0E0EF58FF4F5083CE
:10017000E0917300F0E0EE58FF4F40838AE089B9C8
:100180001092A30088E48AB91CB808958091670092
:1001900081FD26C010BC81E089B988E08AB98AEB6C
:1001A000982F9A95F1F78A95F1F7929AE2E3F0E0A9
:1001B0002DE090E4822F8A95F1F784918CB99BB958
:1001C0005E9BFECF319680E0EA34F80799F71092F3
:1001D0006600929880E98AB98BB390E189278BBB3E
:1001E00008951F920F920FB60F9211242F933F93F1
:1001F0008F939F93AF93BF93EF93FF938BB13CB1DA
:1002000084FF03C05C9881E08BC08091660090E021
:10021000FC013197E830F10508F094C0EF5EFF4F24
:100220000994332361F482E0809366008091A600F4
:100230009091A7009093A5008093A40083C03C3CBC
:1002400009F07EC084E06CC08091A4009091A5006C
:1002500001979093A5008093A400892B09F072C0A8
:1002600083E0809366003093680081E08093A8006B
:1002700069C08091A800E82FF0E0E859FF4F308373
:100280008F5F8093A800883008F45CC08091700074
:1002900081608093700054C0313009F051C080916A
:1002A000670080FD4DC085E08093660083E0809309
:1002B000A8008BB3832713C030937300323308F048
:1002C0003FC0832F90E083539F4F9093A50080936E
:1002D000A40086E0809366008BB392E089278BBBF5
:1002E00031C02091A800E22FF0E0EF58FF4F30839B
:1002F0002F5F2093A8008091A4009091A500830F08
:10030000911D9093A5008093A400809173008217A3
:10031000C9F487E005C08091A500381789F488E00A
:10032000809366000FC08091A400381749F48BB306
:1003300094E089278BBB8091670081608093670080
:1003400010926600FF91EF91BF91AF919F918F91B5
:100350003F912F910F900FBE0F901F9018951F92F5
:100360000F920FB60F9211242F938F939F93EF93B9
:10037000FF938DE08A95F1F72091A300222339F4B1
:1003800091E099B98CEC8CB99093A3001DC0E22F39
:10039000F0E08091730090E001968E179F076CF457
:1003A00082B3805882BB1092660080E98AB9789443
:1003B00080E38A95F1F7929807C0EF58FF4F80814C
:1003C0008CB92F5F2093A300FF91EF919F918F91A4
:1003D0002F910F900FBE0F901F901895CF93DF9322
:1003E0008091670080FF33C1A1E7B0E0C0E6D0E0B4
:1003F000FE0190E030E013962C9113978081281332
:1004000031E02F3F09F091E01196319620E0E63679
:10041000F20789F79111932F992309F013C141E74E
:1004200050E087B161E0862787B910928100309152
:10043000860020E08091870090E0822B932B80350E
:10044000910509F4EAC08135910560F48230910587
:1004500009F444C08330910509F44FC0019709F0B5
:10046000E7C015C08238910509F4A2C08338910510
:1004700028F48036910509F0DBC089C0803F9105E2
:1004800009F469C08050904109F0D2C045C0DA013A
:10049000E0E6F0E058969C9158978081981748F0D4
:1004A000891708F4CFC01196319680E0E636F80738
:1004B00089F7E1E7F0E0968D8881891748F0981771
:1004C00008F4C0C03196219620E0C636D20799F7CD
:1004D0008BB398E089278BBB59DEB4C0809167004D
:1004E0008260809367001092890010928A0082E0F7
:1004F0008093880004DEDC9AA5C0809167008D7F20
:10050000809367001092890010928A0082E08093A5
:100510008800F5DDDC9896C080918500803381F4F9
:1005200080918900813021F480917000826003C045
:10053000809170008D7F809370001092880081C040
:100540008091700081FF03C06093890002C0109207
:10055000890081E06AC080918500803371F46091E8
:100560008A00709189007093A7006093A60081E0D3
:1005700090E043E750E0F0D008C08091A600909151
:10058000A7009093890080938A0082E04EC0CA0140
:1005900048966AE470E043E150E08BD08091A60079
:1005A0009091A700909397008093980083E13DC0BD
:1005B000809185008033F1F480918800813218F0B9
:1005C00080E28093880040918800E199FECF83E02B
:1005D00090E09FBB8EBB4DBB0FB6F894E29AE19AB8
:1005E0000FBE84E090E069E870E050E023E730E07F
:1005F00099D027C0E199FECF83E090E09FBB8EBBEE
:10060000E09A4DB34093880089E890E064E070E0A0
:1006100050E02BE630E056D014C0CA0148966DE594
:1006200070E044E050E045D084E08093880009C049
:100630001092890010928A0082E080938800809353
:1006400081005DDD809167008E7F80936700DF9180
:10065000CF91089581E090E06BE670E04DD09093EB
:10066000A7008093A6008091A6009091A7008150DA
:10067000924030F081E090E09093A7008093A60034
:1006800081B3866081BB9298919A10BC81E089B950
:100690008EE880BD80E98AB91092660080E090E023
:1006A000FC01E859FF4F1082019688309105C1F78F
:1006B0000895FB01DC0102C005900D9241505040AD
:1006C000D8F70895A0E0B0E0E7E6F3E064C07C016D
:1006D000EB018A01690109C0CE012196F601099555
:1006E000F70181937F010150104001151105A1F719
:1006F000CDB7DEB7E8E06BC0DF92EF92FF920F93C9
:100700001F937B018C01FB010995D82EC80101962E
:10071000F7010995982F8D2D1F910F91FF90EF9064
:10072000DF900895A0E0B0E0E7E9F3E034C0EC0129
:100730007B018A01690109C0CE012196F70161910F
:100740007F01F60109950150104001151105A1F72F
:10075000CDB7DEB7E8E03BC0DF92EF92FF920F9398
:100760001F93D72E7A018C01FA010995C8010196D1
:100770006D2DF70109951F910F91FF90EF90DF907C
:1007800008952F923F924F925F926F927F928F9235
:100790009F92AF92BF92CF92DF92EF92FF920F9310
:1007A0001F93CF93DF93CDB7DEB7CA1BDB0B0FB61A
:1007B000F894DEBF0FBECDBF09942A8839884888D7
:1007C0005F846E847D848C849B84AA84B984C8846D
:1007D000DF80EE80FD800C811B81AA81B981CE0F64
:1007E000D11D0FB6F894DEBF0FBECDBFED01089549
:0407F000F894FFCFAB
:0607F400123456880000DB
:00000001FF
